:1000000009C022C021C020C01FC01EC01DC01CC00E
:100010001BC01AC011241FBECFE9CDBF10E0A0E65F
:10002000B0E0E4EBF2E003C0C89531960D92A4363F
:10003000B107D1F710E0A4E6B0E001C01D92A436EC
:10004000B107E1F702D035C1DBCFEF92FF920F93FA
:100050001F93CF93DF93BC9A88D0C92FDD27C7FDAC
:10006000DA95C853DF4F81D0E12C40E4F42EE80E3E
:10007000F91E00E010E015C0C49A77D095958795D9
:100080009595879501960197F1F7C4986ED023E076
:10009000959587952A95E1F701960197F1F70F5FFE
:1000A0001F4F0C171D0741F720E030E0E0E2F0E0C1
:1000B00006C08E2F9F2F0197F1F72F5F3F4F2E1510
:1000C0003F05B9F7C9CFA0E0B0E0E8E6F0E09AC09C
:1000D000D92FC82FA880B980CA80DB80A114B104B1
:1000E000C104D10429F482E49EECACE0BFE132C04B
:1000F0009D2D8C2D7B2D6A2D2DE133EF41E050E0BD
:100100005ED027EA31E440E050E03ED0E62EF72E04
:10011000082F192F9D2D8C2D7B2D6A2D2DE133EF6E
:1001200041E050E04CD0952F842F732F622F24E1B3
:100130003BE040E050E028D0E61AF70A080B190B24
:10014000B12FA02F9F2D8E2D17FF04C081509040FE
:10015000A040B04888839983AA83BB839F77EAE055
:10016000CDB7DEB76BC0AFDF089580E690E0ABDFC0
:100170000895AA27BB278093600090936100A09305
:100180006200B09363000895FF27EE27BB27AA27DC
:1001900060FF04C0A20FB31FE41FF51F220F331F1F
:1001A000441F551F969587957795679589F7009712
:1001B000760771F79F2F8E2F7B2F6A2F089597FB5D
:1001C000092E05260ED057FD04D04CD00AD0001CB5
:1001D00038F450954095309521953F4F4F4F5F4FE4
:1001E0000895F6F790958095709561957F4F8F4FA4
:1001F0009F4F08952F923F924F925F926F927F92FE
:100200008F929F92AF92BF92CF92DF92EF92FF9226
:100210000F931F93CF93DF93CDB7DEB7CA1BDB0BD2
:100220000FB6F894DEBF0FBECDBF09942A88398877
:1002300048885F846E847D848C849B84AA84B9847E
:10024000C884DF80EE80FD800C811B81AA81B9818A
:10025000CE0FD11D0FB6F894DEBF0FBECDBFCA2F93
:10026000DB2F0895A1E21A2EAA1BBB1BEA2FFB2F3E
:100270000DC0AA1FBB1FEE1FFF1FA217B307E40785
:10028000F50720F0A21BB30BE40BF50B661F771FDD
:10029000881F991F1A9469F76095709580959095BD
:1002A000262F372F482F592F6A2F7B2F8E2F9F2FC6
:0402B0000895FFCFDF
:0402B4000100000045
:00000001FF
